******************************************************************************
                  TI ARM Linker PC v5.0.4                      
******************************************************************************
>> Linked Wed Jul 31 15:12:16 2013

OUTPUT FILE NAME:   <Cortex_A15_example_TICC.out>
ENTRY POINT SYMBOL: "Entry"  address: 80005028


MEMORY CONFIGURATION

         name            origin    length      used     unused   attr    fill
----------------------  --------  ---------  --------  --------  ----  --------
  L3                    0c000000   00200000  00000000  00200000  RWIX
  DDR                   80000000   08000000  0080ec44  077f13bc  RWIX


SEGMENT ALLOCATION MAP

run origin  load origin   length   init length attrs members
----------  ----------- ---------- ----------- ----- -------
80000000    80000000    000056e4   000056e4    r-x
  80000000    80000000    000056e4   000056e4    r-x .text
800056e4    800056e4    00001200   00000000    rw-
  800056e4    800056e4    00001200   00000000    rw- .bss
800068e4    800068e4    000001ec   000001ec    rw-
  800068e4    800068e4    000001ec   000001ec    rw- .data
80006ad0    80006ad0    00000174   00000174    r--
  80006ad0    80006ad0    00000174   00000174    r-- .const
80100000    80100000    00804000   00000000    rw-
  80100000    80100000    00004000   00000000    rw- .TTB
  80104000    80104000    00800000   00000000    rw- .sysmem
87ffc000    87ffc000    00004000   00000000    rw-
  87ffc000    87ffc000    00004000   00000000    rw- .stack


SECTION ALLOCATION MAP

 output                                  attributes/
section   page    origin      length       input sections
--------  ----  ----------  ----------   ----------------
.cinit     0    80000000    00000000     UNINITIALIZED

.cinit     0    80000000    00000000     UNINITIALIZED

.init_array 
*          0    80000000    00000000     UNINITIALIZED

.text      0    80000000    000056e4     
                  80000000    0000166c     rtsv7A8_A_le_eabi.lib : _printfi.obj (.text)
                  8000166c    00000924     pktwire.obj (.text)
                  80001f90    00000620     rtsv7A8_A_le_eabi.lib : memory.obj (.text)
                  800025b0    000005d4                           : lowlev.obj (.text)
                  80002b84    000004d8                           : trgdrv.obj (.text)
                  8000305c    00000484     cp15.obj (.text)
                  800034e0    000002d8     rtsv7A8_A_le_eabi.lib : fopen.obj (.text)
                  800037b8    000002b8                           : ull_div32.obj (.text)
                  80003a70    00000214                           : fd_add32.obj (.text)
                  80003c84    000001c8                           : fputs.obj (.text)
                  80003e4c    00000190                           : fd_div32.obj (.text)
                  80003fdc    00000180                           : memcpy32.obj (.text)
                  8000415c    0000016c     mmu.obj (.text)
                  800042c8    00000154     v7_pmu.obj (.text)
                  8000441c    00000148     rtsv7A8_A_le_eabi.lib : setvbuf.obj (.text)
                  80004564    00000134     cache.obj (.text)
                  80004698    00000128     rtsv7A8_A_le_eabi.lib : fd_mul32.obj (.text)
                  800047c0    00000118                           : _io_perm.obj (.text)
                  800048d8    00000118                           : fflush.obj (.text)
                  800049f0    00000118                           : i_div32.obj (.text)
                  80004b08    00000104                           : fputc.obj (.text)
                  80004c0c    000000f4                           : u_div32.obj (.text)
                  80004d00    000000d4                           : auto_init.obj (.text)
                  80004dd4    000000d4                           : fclose.obj (.text)
                  80004ea8    000000d0                           : fd_cmp32.obj (.text)
                  80004f78    000000b0                           : memset32.obj (.text)
                  80005028    000000ac     init.obj (.text)
                  800050d4    000000a8     rtsv7A8_A_le_eabi.lib : fseek.obj (.text)
                  8000517c    000000a8                           : trgmsg.obj (.text)
                  80005224    000000a4                           : printf.obj (.text)
                  800052c8    00000084                           : atoi.obj (.text)
                  8000534c    00000084                           : xdtest.obj (.text)
                  800053d0    00000080                           : cpy_tbl.obj (.text)
                  80005450    00000080                           : ltoa.obj (.text)
                  800054d0    0000005c                           : fd_toi32.obj (.text)
                  8000552c    00000048                           : strncpy.obj (.text)
                  80005574    0000003c                           : i_tofd32.obj (.text)
                  800055b0    0000002c                           : memccpy.obj (.text)
                  800055dc    0000002c                           : memchr.obj (.text)
                  80005608    00000028                           : strchr.obj (.text)
                  80005630    00000028                           : strcmp.obj (.text)
                  80005658    00000024                           : _lock.obj (.text)
                  8000567c    00000020                           : icall32.obj (.text)
                  8000569c    0000001c                           : strlen.obj (.text)
                  800056b8    00000018                           : strcpy.obj (.text)
                  800056d0    00000014                           : xdclass.obj (.text)

.bss       0    800056e4    00001200     UNINITIALIZED
                  800056e4    00001000     pktwire.obj (.bss:testdata)
                  800066e4    00000120     rtsv7A8_A_le_eabi.lib : trgmsg.obj (.bss:__CIOBUF_)
                  80006804    000000a0                           : defs.obj (.bss:_tmpnams)
                  800068a4    00000028     pktwire.obj (.bss:testcycle)
                  800068cc    00000010     pktwire.obj (.bss)
                  800068dc    00000008     rtsv7A8_A_le_eabi.lib : trgdrv.obj (.bss)

.data      0    800068e4    000001ec     
                  800068e4    000000f0     rtsv7A8_A_le_eabi.lib : defs.obj (.data:_ftable)
                  800069d4    000000cc                           : lowlev.obj (.data)
                  80006aa0    00000010                           : defs.obj (.data)
                  80006ab0    0000000c                           : memory.obj (.data)
                  80006abc    00000008                           : _lock.obj (.data)
                  80006ac4    00000008                           : exit.obj (.data)
                  80006acc    00000004                           : fopen.obj (.data)

.const     0    80006ad0    00000174     
                  80006ad0    00000101     rtsv7A8_A_le_eabi.lib : ctype.obj (.const:.string:_ctypes_)
                  80006bd1    00000003     --HOLE-- [fill = 0]
                  80006bd4    00000070     pktwire.obj (.const)

.TTB       0    80100000    00004000     UNINITIALIZED
                  80100000    00004000     pktwire.obj (.TTB)

.sysmem    0    80104000    00800000     UNINITIALIZED
                  80104000    00000008     rtsv7A8_A_le_eabi.lib : memory.obj (.sysmem)
                  80104008    007ffff8     --HOLE--

.stack     0    87ffc000    00004000     UNINITIALIZED
                  87ffc000    00004000     --HOLE--


GLOBAL SYMBOLS: SORTED ALPHABETICALLY BY Name 

address    name
--------   ----
800051c4   C$$IO$$
800034b4   CP15AuxControlFeatureDisable
800034a0   CP15AuxControlFeatureEnable
80003440   CP15BranchPredictionDisable
80003430   CP15BranchPredictionEnable
80003424   CP15BranchPredictorInvalidate
80003460   CP15ControlFeatureDisable
80003474   CP15ControlFeatureEnable
8000313c   CP15DCacheClean
80003274   CP15DCacheCleanBuff
800031d0   CP15DCacheCleanFlush
800032c8   CP15DCacheCleanFlushBuff
8000306c   CP15DCacheDisable
80003098   CP15DCacheEnable
800030a8   CP15DCacheFlush
8000331c   CP15DCacheFlushBuff
80003450   CP15DomainAccessClientSet
8000305c   CP15ICacheDisable
80003088   CP15ICacheEnable
80003264   CP15ICacheFlush
80003380   CP15ICacheFlushBuff
800033ec   CP15MMUDisable
80003404   CP15MMUEnable
800034c8   CP15MainIdPrimPartNumGet
800033e0   CP15TlbInvalidate
800033d4   CP15Ttb0Set
80003488   CP15TtbCtlTtb0Config
80003418   CP15VectorBaseAddrSet
8000462c   CacheDataCleanAll
80004644   CacheDataCleanBuff
80004620   CacheDataCleanInvalidateAll
8000467c   CacheDataCleanInvalidateBuff
80004638   CacheDataInvalidateAll
80004660   CacheDataInvalidateBuff
80004564   CacheDisable
800045ac   CacheEnable
800045f8   CacheInstInvalidateAll
80004604   CacheInstInvalidateBuff
80005028   Entry
80002fec   HOSTclock
80002f84   HOSTclose
80002f1c   HOSTgetenv
80002e78   HOSTlseek
80002dec   HOSTopen
80002d68   HOSTread
80002cd0   HOSTrename
80002c6c   HOSTtime
80002c08   HOSTunlink
80002b84   HOSTwrite
8000567c   IND_CALL
800016f8   MMUConfigAndEnable
800042ac   MMUEnable
8000415c   MMUInit
800041bc   MMUMemRegionMap
UNDEFED    SHT$$INIT_ARRAY$$Base
UNDEFED    SHT$$INIT_ARRAY$$Limit
800056d0   _Dclass
8000534c   _Dtest
800066e4   __CIOBUF_
88000000   __STACK_END
00004000   __STACK_SIZE
00800000   __SYSMEM_SIZE
UNDEFED    __TI_CINIT_Base
UNDEFED    __TI_CINIT_Limit
UNDEFED    __TI_Handler_Table_Base
00000001   __TI_args_main
80004d00   __TI_auto_init
80000000   __TI_static_base__
80004ea8   __aeabi_cdcmpeq
80004ea8   __aeabi_cdcmple
800054d0   __aeabi_d2iz
80003a7c   __aeabi_dadd
80003e4c   __aeabi_ddiv
80004698   __aeabi_dmul
80003a70   __aeabi_dsub
80005574   __aeabi_i2d
800049f0   __aeabi_idivmod
80004f78   __aeabi_memclr
80004f78   __aeabi_memclr4
80004f78   __aeabi_memclr8
80003fdc   __aeabi_memcpy
80003fdc   __aeabi_memcpy4
80003fdc   __aeabi_memcpy8
80004f7c   __aeabi_memset
80004f7c   __aeabi_memset4
80004f7c   __aeabi_memset8
80006aac   __aeabi_stderr
80006aa4   __aeabi_stdin
80006aa8   __aeabi_stdout
80004c0c   __aeabi_uidivmod
800037b8   __aeabi_uldivmod
ffffffff   __binit__
ffffffff   __c_args__
87ffc000   __stack
800042ec   _ccnt_divider
80003620   _cleanup
80006ac4   _cleanup_ptr
80004dd4   _closefile
80006ad0   _ctypes_
80004330   _disable_ccnt
800043d0   _disable_ccnt_irq
8000434c   _disable_pmn
800043ec   _disable_pmn_irq
80004314   _disable_pmu
80004370   _disable_pmu_user_access
800048d8   _doflush
80006ac8   _dtors_ptr
80004324   _enable_ccnt
800043c4   _enable_ccnt_irq
8000433c   _enable_pmn
800043dc   _enable_pmn_irq
80004304   _enable_pmu
8000435c   _enable_pmu_user_access
80006aa0   _ft_end
800068e4   _ftable
800042c8   _getPMN
80006abc   _lock
80005670   _nop
800042d8   _pmn_config
800043a0   _pmu_software_increment
80001168   _printfi
80004860   _rd_ok
80004384   _read_ccnt
800043b0   _read_flags
8000438c   _read_pmn
80005664   _register_lock
80005658   _register_unlock
8000440c   _reset_ccnt
800043fc   _reset_pmn
80104000   _sys_memory
80006804   _tmpnams
80006ac0   _unlock
800043b8   _write_flags
800047c0   _wrt_ok
80002a88   add_device
800052c8   atoi
ffffffff   binit
800068e4   bss_end
800056e4   bss_start
800068d0   bufPtr
8000254c   calloc
800029f8   close
800053d0   copy_in
800068d4   descLen
80004e68   fclose
8000495c   fflush
800036b8   fopen
80004b08   fputc
80003c84   fputs
8000213c   free
8000366c   freopen
800050d4   fseek
800068cc   hostDesc
80002980   lseek
80005450   ltoa
800019d8   main
80002088   malloc
80002414   memalign
800055b0   memccpy
800055dc   memchr
80003fdc   memcpy
80004f88   memset
80001f90   minit
800028a4   open
8000522c   printf
80004bf4   putc
80004bf8   putchar
80003e14   puts
800027dc   read
800051cc   readmsg
80002290   realloc
800026e0   remove
80002790   remove_device
80002724   rename
8000441c   setvbuf
80005608   strchr
80005630   strcmp
800056b8   strcpy
8000569c   strlen
8000552c   strncpy
8000166c   testcode
800068a4   testcycle
800068d8   testcycle_tmp
800056e4   testdata
800026e0   unlink
800025b0   write
8000517c   writemsg


GLOBAL SYMBOLS: SORTED BY Symbol Address 

address    name
--------   ----
00000001   __TI_args_main
00004000   __STACK_SIZE
00800000   __SYSMEM_SIZE
80000000   __TI_static_base__
80001168   _printfi
8000166c   testcode
800016f8   MMUConfigAndEnable
800019d8   main
80001f90   minit
80002088   malloc
8000213c   free
80002290   realloc
80002414   memalign
8000254c   calloc
800025b0   write
800026e0   remove
800026e0   unlink
80002724   rename
80002790   remove_device
800027dc   read
800028a4   open
80002980   lseek
800029f8   close
80002a88   add_device
80002b84   HOSTwrite
80002c08   HOSTunlink
80002c6c   HOSTtime
80002cd0   HOSTrename
80002d68   HOSTread
80002dec   HOSTopen
80002e78   HOSTlseek
80002f1c   HOSTgetenv
80002f84   HOSTclose
80002fec   HOSTclock
8000305c   CP15ICacheDisable
8000306c   CP15DCacheDisable
80003088   CP15ICacheEnable
80003098   CP15DCacheEnable
800030a8   CP15DCacheFlush
8000313c   CP15DCacheClean
800031d0   CP15DCacheCleanFlush
80003264   CP15ICacheFlush
80003274   CP15DCacheCleanBuff
800032c8   CP15DCacheCleanFlushBuff
8000331c   CP15DCacheFlushBuff
80003380   CP15ICacheFlushBuff
800033d4   CP15Ttb0Set
800033e0   CP15TlbInvalidate
800033ec   CP15MMUDisable
80003404   CP15MMUEnable
80003418   CP15VectorBaseAddrSet
80003424   CP15BranchPredictorInvalidate
80003430   CP15BranchPredictionEnable
80003440   CP15BranchPredictionDisable
80003450   CP15DomainAccessClientSet
80003460   CP15ControlFeatureDisable
80003474   CP15ControlFeatureEnable
80003488   CP15TtbCtlTtb0Config
800034a0   CP15AuxControlFeatureEnable
800034b4   CP15AuxControlFeatureDisable
800034c8   CP15MainIdPrimPartNumGet
80003620   _cleanup
8000366c   freopen
800036b8   fopen
800037b8   __aeabi_uldivmod
80003a70   __aeabi_dsub
80003a7c   __aeabi_dadd
80003c84   fputs
80003e14   puts
80003e4c   __aeabi_ddiv
80003fdc   __aeabi_memcpy
80003fdc   __aeabi_memcpy4
80003fdc   __aeabi_memcpy8
80003fdc   memcpy
8000415c   MMUInit
800041bc   MMUMemRegionMap
800042ac   MMUEnable
800042c8   _getPMN
800042d8   _pmn_config
800042ec   _ccnt_divider
80004304   _enable_pmu
80004314   _disable_pmu
80004324   _enable_ccnt
80004330   _disable_ccnt
8000433c   _enable_pmn
8000434c   _disable_pmn
8000435c   _enable_pmu_user_access
80004370   _disable_pmu_user_access
80004384   _read_ccnt
8000438c   _read_pmn
800043a0   _pmu_software_increment
800043b0   _read_flags
800043b8   _write_flags
800043c4   _enable_ccnt_irq
800043d0   _disable_ccnt_irq
800043dc   _enable_pmn_irq
800043ec   _disable_pmn_irq
800043fc   _reset_pmn
8000440c   _reset_ccnt
8000441c   setvbuf
80004564   CacheDisable
800045ac   CacheEnable
800045f8   CacheInstInvalidateAll
80004604   CacheInstInvalidateBuff
80004620   CacheDataCleanInvalidateAll
8000462c   CacheDataCleanAll
80004638   CacheDataInvalidateAll
80004644   CacheDataCleanBuff
80004660   CacheDataInvalidateBuff
8000467c   CacheDataCleanInvalidateBuff
80004698   __aeabi_dmul
800047c0   _wrt_ok
80004860   _rd_ok
800048d8   _doflush
8000495c   fflush
800049f0   __aeabi_idivmod
80004b08   fputc
80004bf4   putc
80004bf8   putchar
80004c0c   __aeabi_uidivmod
80004d00   __TI_auto_init
80004dd4   _closefile
80004e68   fclose
80004ea8   __aeabi_cdcmpeq
80004ea8   __aeabi_cdcmple
80004f78   __aeabi_memclr
80004f78   __aeabi_memclr4
80004f78   __aeabi_memclr8
80004f7c   __aeabi_memset
80004f7c   __aeabi_memset4
80004f7c   __aeabi_memset8
80004f88   memset
80005028   Entry
800050d4   fseek
8000517c   writemsg
800051c4   C$$IO$$
800051cc   readmsg
8000522c   printf
800052c8   atoi
8000534c   _Dtest
800053d0   copy_in
80005450   ltoa
800054d0   __aeabi_d2iz
8000552c   strncpy
80005574   __aeabi_i2d
800055b0   memccpy
800055dc   memchr
80005608   strchr
80005630   strcmp
80005658   _register_unlock
80005664   _register_lock
80005670   _nop
8000567c   IND_CALL
8000569c   strlen
800056b8   strcpy
800056d0   _Dclass
800056e4   bss_start
800056e4   testdata
800066e4   __CIOBUF_
80006804   _tmpnams
800068a4   testcycle
800068cc   hostDesc
800068d0   bufPtr
800068d4   descLen
800068d8   testcycle_tmp
800068e4   _ftable
800068e4   bss_end
80006aa0   _ft_end
80006aa4   __aeabi_stdin
80006aa8   __aeabi_stdout
80006aac   __aeabi_stderr
80006abc   _lock
80006ac0   _unlock
80006ac4   _cleanup_ptr
80006ac8   _dtors_ptr
80006ad0   _ctypes_
80104000   _sys_memory
87ffc000   __stack
88000000   __STACK_END
ffffffff   __binit__
ffffffff   __c_args__
ffffffff   binit
UNDEFED    SHT$$INIT_ARRAY$$Base
UNDEFED    SHT$$INIT_ARRAY$$Limit
UNDEFED    __TI_CINIT_Base
UNDEFED    __TI_CINIT_Limit
UNDEFED    __TI_Handler_Table_Base

[187 symbols]
